:020000040000FA
:0400000023EF00F0FA
:040008003EEF24F0B3
:080018009E928150E76E0D4B32
:1000200004D00E19D8B411000E1B0D51DF6ED92A61
:100030000D6BE12AE950E162110035EC01F0E106B7
:10004000D90602811100D86AF26A9E6AF16AF06AE2
:10005000FA6AFB6A0F01D08E026B070EC16E806ACE
:10006000816A826A808AF19E0F0E926EFF0E936EF5
:10007000BF0E946E030E1F6F040E206FA1EC01F0F3
:10008000150E82B8040EAF6E240EAC6E900EAB6EE1
:10009000B86A106B116B126B136B146B156B166BCC
:1000A0000F6B9EBA08D00F2B0FAB808A0FBB809AC4
:1000B000A1EC01F0F6D7AE50046F39EC01F0045119
:1000C000490AD8B4BFEF01F004514A0AD8B4AFEFDF
:1000D00002F00451570AD8B4D8EF01F00451580A7D
:1000E000D8B4DEEF01F00451590AD8B4E2EF01F0C0
:1000F00004515A0AD8B4A9EF01F00451440AD8B403
:10010000B4EF01F004513F0A27E00451300A72E0D5
:100110000451310A73E00451320A74E00451330A85
:1001200075E00451340A66E00451350A67E0045171
:10013000360A68E00451370A69E00451380A6AE077
:100140000451530AD8B48AEF24F00451560AD8B4A3
:100150000DEF26F051EF00F0330E39EC01F0360EC2
:1001600039EC01F051EF00F09EAA0AD0AE50390AE6
:1001700007E135EC01F0390E39EC01F051EF00F0F8
:10018000E150E95C13E0010EEA6EEF50006F020EE1
:10019000EA6EEF50016FE92A02BBD4EF00F002A330
:1001A0006ED802B385D8E0D7A3D8DED702A1DCD7BA
:1001B000FE0E166F9EAA0AD0AE50390AE1E135EC68
:1001C00001F0390E39EC01F051EF00F0010EEA6E4A
:1001D000EF50006F020EEA6EEF50016FE92A02A3A2
:1001E0004ED802B365D8162FE5D7FF0E39EC01F0D3
:1001F00051EF00F0130E0C6F18D8B6D7310E0C6FFC
:1002000014D8B2D7630E0C6F10D8AED7C70E0C6FD0
:100210000CD8AAD7630E0C6F01D8A6D7808A02919A
:100220000293028B1A6B1B6B08D0808A0291029B8F
:100230000293340E045DD8A8028301EE00F011EEA3
:1002400000F022EE00F00D6B02918150FF0A0E6F5C
:10025000CA6ACC6AF26A9D6A9E6A9F920C51CB6E02
:100260009D82F28CF28ECA841200CA84F26A809A4D
:10027000120082BAFED79EA8FED7AD6E12000151C1
:10028000C00B036F03430341300B8009036F005120
:100290000F0B031182BAFED79EA8FED7AD6E015197
:1002A0003F0B400982BAFED79EA8FED7AD6E120062
:1002B0000151C00B036F03430341300B8009036FEF
:1002C00000390C0B031182BAFED79EA8FED7AD6E83
:1002D00000513F0B82BAFED79EA8FED7AD6E0151EA
:1002E0003F0B400982BAFED79EA8FED7AD6E120022
:1002F00001510DE0400E01610AD001470145036F35
:100300000051030B1C6F03118EEC01F012001C5105
:100310008EEC01F0400E015FEDE112001A2782BA67
:10032000FED79EA8FED7AD6E1B2B1BA712001A513D
:100330007F0B82BAFED79EA8FED7AD6E1B6B1A6BE1
:100340001200830E046F056F042FFED7052FFCD714
:1003500012001FEE10F0040E18D8D8A051EF00F0D4
:10036000106B126B51EF00F01FEE14F0020E0DD85F
:10037000D8A051EF00F0146B156B51EF00F01FEE99
:1003800019F0010E02D851EF00F0808A036F320E8F
:100390000F6F9EBA06D0A1EC01F00F2FFAD7D880CC
:1003A0001200AE50E66E65DF032FF1D7D890120031
:1003B000106B126B0295029751EF00F002950287C5
:1003C00051EF00F00285029751EF00F0165151DF16
:1003D0000F0E4FDF000E4DDF10EE00F0E65049DF4C
:1003E000E150D8B4A1EC01F00F0EE262F7D7120091
:1003F000D89002A51200105117E111510AE082A60F
:1004000003D09EAAFCD722D082B612009EAAFCD7A7
:100410001DD082B603D09EAAFCD718D082A629EFA1
:1004200002F09EAAFBD712D081501015111903E0DB
:100430009EAAFAD70BD01251D8B429EF02F081143A
:100440001319D8B429EF02F09EAAF5D7D880AE5080
:10045000120014511519D8B4120000001407143DED
:10046000152B150714511511D8A4F7D7D8901200E1
:10047000162B1051D8B4010C10EE00F00A0EE262F7
:1004800004D09EAA000CAE50020C1051E614E652A5
:100490001119D8A4F3D71251D8B4010CE7141319C9
:1004A000D8A4ECD7010C162B1051D8B4010C10EEC7
:1004B00000F00A0EE26204D09EAA000CAE50020CBC
:1004C0001051E6141119D8A4F4D71251D8B4010C64
:1004D000E7141319D8A4EDD7010C162B1051D8B47A
:1004E000010C10EE00F0E7380F0B186F02890A0EAE
:1004F000E26204D09EAA000CAE50020C1851176F95
:1005000002A905D00299E6500F0B186F04D002899A
:10051000E7380F0B186F105117151119D8A4E7D72A
:100520001251D8B4010C18151319D8A4E0D7010C36
:1005300000000000000000000000000000000000BB
:1005400000000000000000000000000000000000AB
:10055000000000000000000000000000010C050E7B
:10056000FA6E1947194519437C0BF92651EF00F033
:1005700051EF00F044EF04F026EF03F032EF03F008
:1005800032EF03F051EF00F051EF00F051EF00F0C7
:100590009CEF04F01CEF04F00EEF03F01AEF03F0F1
:1005A0001AEF03F051EF00F051EF00F0CCEF04F040
:1005B0007EEF04F0FBEF03F0F6EF02F002EF03F042
:1005C00002EF03F051EF00F051EF00F051EF00F0B7
:1005D00051EF00F051EF00F051EF00F051EF00F05B
:1005E00051EF00F051EF00F051EF00F0808A0291DE
:1005F000166BFEDED8B051EF00F019AF3EEF03F0FE
:10060000E7EF22F0808A0291166BF2DED8B051EF4C
:1006100000F019AF3EEF03F088EF23F0808A0291DB
:10062000166BE6DED8B051EF00F019AF67EF03F0BC
:100630001BEF23F0808A0291166BDADED8B051EFFF
:1006400000F019AF67EF03F0C4EF23F0808A029146
:10065000166BCEDED8B051EF00F019AFA6EF03F065
:1006600051EF23F0808A0291166BC2DED8B051EFB1
:1006700000F019AFA6EF03F006EF24F010EE00F043
:1006800081CFE6FF13D80F0EE262FAD702A751EF2F
:1006900003F053EC02F0010A04E0010AEFE051EF2D
:1006A00000F0E6EC01F0809A51EF00F01951070BD1
:1006B000030A08E01951070B040A02E0E60E03D012
:1006C000F70E01D0FF0E010FFEE100D0120010EE78
:1006D00000F08138F00BE76E18D881500F0BE7104F
:1006E000E66E24D80F0EE262F4D702A780EF03F083
:1006F0006DEC02F0010A04E0010AE9E051EF00F0BC
:10070000E6EC01F0809A51EF00F01951070B030A53
:1007100008E01951070B040A02E0E50E03D0F60EBB
:1007200001D0FE0E010FFEE100D012001951070B9F
:10073000030A08E01951070B040A02E0E60E03D091
:10074000F70E01D0FF0E010FFEE1120010EE00F0D7
:1007500081CF03FF0333E7320333E73228D881CF59
:1007600003FF0333E7320333E73221D881CF03FF9E
:100770000333E7320333E7321AD881CF03FF033361
:10078000E7320333E63224D80F0EE262E1D702A744
:10079000D2EF03F098EC02F0010A04E0010AD6E07F
:1007A00051EF00F0E6EC01F0809A51EF00F01951A2
:1007B000070B030A08E01951070B040A02E0E60ED2
:1007C00003D0F70E01D0FF0E010FFEE100D01200A2
:1007D0001951070B030A0AE01951070B040A03E039
:1007E000E70E000005D0F80E000002D00000120055
:1007F000010FFEE11200808A0291166BF9DDD8B07C
:1008000051EF00F010EE00F00F0E81CFE6FF000078
:1008100000D000D0E262F9D702A717EF04F053EC42
:1008200002F0010A04E0010AEDE051EF00F0E6EC0D
:1008300001F0809A51EF00F0808A0291166BD8DDAA
:10084000D8B051EF00F010EE00F08138F00BE76EF9
:10085000000000D000D000D081500F0BE710E66EF2
:100860000F0E00D0E262F1D702A73FEF04F06DEC6B
:1008700002F0010A04E0010AE6E051EF00F0E6ECC4
:1008800001F0809A51EF00F0808A0291166BB0DD82
:10089000D8B051EF00F010EE00F081CF03FF03332A
:1008A000E7320333E73200D000D081CF03FF0333B8
:1008B000E7320333E73200D000D081CF03FF0333A8
:1008C000E7320333E73200D000D081CF03FF033398
:1008D000E7320333E6320F0EE262DFD702A779EF89
:1008E00004F098EC02F0010A04E0010AD4E051EFB0
:1008F00000F0E6EC01F0809A51EF00F0808A02915E
:10090000166B76DDD8B051EF00F010EE00F00F0E50
:1009100081CFE6FFE262FCD702A797EF04F053EC29
:1009200002F0010A04E0010AF0E051EF00F0E6EC09
:1009300001F0809A51EF00F0808A0291166B58DD29
:10094000D8B051EF00F010EE00F020EE00F001EE14
:1009500000F08138F00BE76E0F0EDE528114E612C4
:10096000DAA6F7D700008138F00BE76E0F0EEE52D3
:100970008114E612EAA6F7D702A7C7EF04F06DECE0
:1009800002F0010A04E0010ADEE051EF00F0E6ECBB
:1009900001F0809A51EF00F0808A0291166B28DDF9
:1009A000D8B051EF00F010EE00F081CFE6FF81CF1C
:1009B000E6FF81CFE6FF81CFE6FF81CFE6FF81CF63
:1009C000E6FF81CFE6FF81CFE6FF81CFE6FF81CF53
:1009D000E6FF81CFE6FF81CFE6FF81CFE6FF81CF43
:1009E000E6FF81CFE6FF81CFE6FF81CFE6FF81CF33
:1045A000E6FF81CFE6FF81CFE6FF02A7E2EF22F030
:1045B00053EC02F0010A06E0010AD8B4D3EF04F08C
:1045C00051EF00F0E6EC01F0809A51EF00F010EEB0
:1045D00000F081500E6F0D6BE66EE66A81500D4B58
:1045E0001ED00E19D8B420D00E1B0E5100D000D012
:1045F000E66E0D51E66E0D6B0F0EE262EFD702A76D
:104600000AEF23F038EC02F0010A04E0010ADFE0CF
:1046100051EF00F0E6EC01F0809A51EF00F00E6FE0
:1046200000D000D00000E4D700D000D000D000D0EF
:1046300000D00000D3D70F0E1D6F10EE00F0815098
:104640001D150E6F0D6BE66E81501D150D2B0DB9EE
:104650001DD00E19D8B41FD00E1B0D39F00B0E1142
:1046600000D0E66E0D6B0F0EE262EED702A741EFAF
:1046700023F053EC02F0010A04E0010ADEE051EFFE
:1046800000F0E6EC01F0809A51EF00F00E6F00D0E0
:1046900000D00000E6D700D000D000D000D000004D
:1046A000D3D7030E1D6F10EE00F081501D150E6F55
:1046B0000D6BE66E81501D150D2B0DBD1ED00E1914
:1046C000D8B420D00E1B0D470D45FC0B0E11000079
:1046D000E66E0D6B0F0EE262EDD702A778EF23F0C6
:1046E00053EC02F0010A04E0010ADDE051EF00F0B2
:1046F000E6EC01F0809A51EF00F00E6F00D000D090
:104700000000E6D700D000D000D000D00000D2D703
:1047100010EE00F081500E6F0D6BE66EE66A815070
:104720000D4B1DD00E19D8B41DD00E1B21D80E5123
:10473000E66E0D51E66E0D6B0F0EE262F0D702A72A
:10474000AAEF23F038EC02F0010A04E0010AE0E0ED
:1047500051EF00F0E6EC01F0809A51EF00F00E6F9F
:1047600007D8E5D700D000D000D0000001D8D7D7B7
:104770001951070B040A03E0E80E00D002D0F80E2E
:104780000000010FFEE112000F0E1D6F10EE00F091
:1047900081501D150E6F0D6BE66E81501D150D2B92
:1047A0000DB91ED00E19D8B41FD00E1B23D80D3949
:1047B000F00B0E110000E66E0D6B0F0EE262EDD7EE
:1047C00002A7EBEF23F053EC02F0010A04E0010A28
:1047D000DDE051EF00F0E6EC01F0809A51EF00F0DF
:1047E0000E6FC6DF0E51E7D700D000D000D000D04A
:1047F00001D8D3D71951070B040A03E0E90E00D002
:1048000002D0F90E0000010FFEE11200030E1D6F31
:1048100010EE00F081501D150E6F0D6BE66E81508D
:104820001D150D2B0DBD1ED00E19D8B421D00E1B99
:10483000E1DF0D470D45FC0B0E11E66E0D6B0F0E03
:10484000E262EDD702A72DEF24F053EC02F0010A4B
:1048500004E0010ADDE051EF00F0E6EC01F0809A9F
:1048600051EF00F00E6FC6DF0E5100D00000E5D70B
:1048700000D000D000D000D0BDDFD1D79E92811CE7
:104880002C6F346F343332B12133343332B32233AB
:10489000343332B52333343332B72433343332B97B
:1048A0002533343332BB2633343332BD27333433EC
:1048B00032BF2833343132152D132E512F112C15C0
:1048C0003311356F2C1D2F153211366F32512915CA
:1048D0002B132D1D3115326F335129132C1D331518
:1048E0002A1331512D15336F311D2D173051316F72
:1048F0002C1D2E152F6F35512E6F3651306F1F51D5
:104900002917110070B8498A70B8488A10E608ADB6
:1049100000AD0056808A01EE00F011EE00F0029129
:10492000800E216F226F236F246F256F266F276FF4
:10493000286F296B2A6B2D6BFF0E2E6F2F6B306B40
:10494000316B326B336B0F0E1E6FF86A490EF76EC8
:10495000040EF66E20450E0BF626CA6ACC6AF26A81
:104960009D6A9E6A9F820900F550CA6E0900F55043
:10497000CB6E9D82F28CF28ECA849EAA0AD0AE5073
:10498000390A07E135EC01F0390E39EC01F051EF4D
:1049900000F029B120D829B341D829B562D829B768
:1049A00083D829B9A4D829BBC5D829BDE6D829BF41
:1049B00007D982BAE2D79EA8E0D7E150E95C04E0CB
:1049C000EF50AD6EE92AD9D702A1D7D7FF0E39EC47
:1049D00001F051EF00F02AB10FD02BB116D0000E2C
:1049E0001E1904E0000E1E6F80090DD921510BD94C
:1049F0002991800E216F12002A912991000E1E6FBD
:104A0000C00901D9800E216F12002B912991000E4F
:104A10001E6FA009F8D8800E216F12002AB30FD0A4
:104A20002BB316D0010E1E1904E0010E1E6F800973
:104A3000EAD82251E8D82993800E226F12002A93D7
:104A40002993010E1E6FC009DED8800E226F12005E
:104A50002B932993010E1E6FA009D5D8800E226FCB
:104A600012002AB50FD02BB516D0020E1E1904E085
:104A7000020E1E6F8009C7D82351C5D82995800E14
:104A8000236F12002A952995020E1E6FC009BBD80C
:104A9000800E236F12002B952995020E1E6FA00920
:104AA000B2D8800E236F12002AB70FD02BB716D0C2
:104AB000030E1E1904E0030E1E6F8009A4D82451B2
:104AC000A2D82997800E246F12002A972997030EE7
:104AD0001E6FC00998D8800E246F12002B9729975B
:104AE000030E1E6FA0098FD8800E246F12002AB902
:104AF0000FD02BB916D0040E1E1904E0040E1E6F41
:104B0000800981D825517FD82999800E256F120000
:104B10002A992999040E1E6FC00975D8800E256F39
:104B200012002B992999040E1E6FA0096CD8800ED3
:104B3000256F12002ABB0FD02BBB16D0050E1E19F5
:104B400004E0050E1E6F80095ED826515CD8299BB3
:104B5000800E266F12002A9B299B050E1E6FC0092E
:104B600052D8800E266F12002B9B299B050E1E6FBC
:104B7000A00949D8800E266F12002ABD0FD02BBD88
:104B800016D0060E1E1904E0060E1E6F80093BD8D3
:104B9000275139D8299D800E276F12002A9D299D03
:104BA000060E1E6FC0092FD8800E276F12002B9D96
:104BB000299D060E1E6FA00926D8800E276F1200B1
:104BC0002ABF0FD02BBF16D0070E1E1904E0070E08
:104BD0001E6F800918D8285116D8299F800E286F7B
:104BE00012002A9F299F070E1E6FC0090CD8800E45
:104BF000286F12002B9F299F070E1E6FA00903D854
:104C0000800E286F1200E76EE12AE950E16212007F
:104C100035EC01F0E106028112001FEE1FF0020EDA
:104C2000C5EC01F0D8A051EF00F0030E1F6F040E89
:064C3000206F51EF00F0BF
:020000040030CA
:03000100061A0ECE
:020005008181F7
:060008000FC00FE00F40E5
:00000001FF
